:100000000C9497050C94DF050C94DF050C94DF0528
:100010000C94DF050C94DF050C94DF050C94DF05D0
:100020000C94DF050C94DF050C94FD0F0C94DF0598
:100030000C94111E0C94DF050C94DF050C94DF0565
:100040000C94DF050C94DF050C94DF050C94DF05A0
:100050000C94DF050C946A1E0C94DF050C94DF05EC
:100060000C94DF050C9476080C94DF050C94DF05E6
:100070000C94DF050C94DF050C94DF050C94DF0570
:100080000C94DF050C94DF050C94DF050C94DF0560
:100090000C94DF050C94DF050C94DF050C94DF0550
:1000A0000C94DF050C94DF050C94DF054B0E720EEB
:1000B0006A0F720E6A0FBE0EE10E6A0F380F470FFD
:1000C000451445147D147D14F8142C15231723179B
:1000D00043152317D414D414DD162317F216101762
:1000E0008800000000000000040005000600070072
:1000F000080009000A000B000C000D000E000F00A4
:100100001000110012001300140015001600170053
:10011000180019001A001B001C001D001E001F0003
:1001200020002100220023002400250026002700B3
:10013000280029002A002B002C002D002E002F0063
:10014000300031000000330034000000360037007A
:10015000380082003A003B003C003D003E003F007A
:1001600040004100420043004400450046000000BA
:10017000000049004A004E004C004D004B004F006B
:100180005000510052000000540055005600570026
:10019000580059005A005B005C005D005E005F0083
:1001A0006000610062006300000065008500670078
:1001B000680069006A000000000000000000000004
:1001C0000000000000000000890087008A008B000A
:1001D000E000E100E200E3000000E500E600E700E7
:1001E000291E1F20212223242526272D2E742A2B69
:1001F000141A0815171C180C12132F302804160790
:10020000090A0B0D0E0F3334311D1B061905111091
:10021000363738752C764E4B494C52504F514A4D1B
:1002200056545F6061555C5D5E57595A5B67626604
:100230006377444568696A807071727380806580F5
:1002400048463A3B3C3D3E3F4041424380808080AF
:100250007939007A7880807B7F7E8080807D808085
:10026000706339385F6C65643A20253032580A0073
:100270007573625F6C65643A20253032580A0073EA
:10028000656E6420253032583A20253032580A00F5
:1002900073656E642039443A20253032580A007262
:1002A00025303258200073656E642037303A20259F
:1002B0003032580A0073656E642039433A20253085
:1002C00032580A00722530345820007325303258D5
:1002D00020006F6C6420747970650A006E65772069
:1002E000747970650A000A4B6579626F61726420E7
:1002F00073746172742E0A000A55534220636F6E44
:10030000666967757265642E0A000A0A544D4B3A95
:1003100064373362656462352F4C5546410A0A00E2
:100320003003500043003900380020006B006500A6
:10033000790062006F0061007200640020006300B9
:100340006F006E0076006500720074006500720038
:1003500000000E0374002E006D002E006B002E00B6
:1003600000000403090409027400040100A032091A
:1003700004000001030101000921110100012240D4
:10038000000705810308000A0904010001030102B6
:1003900000092111010001224D0007058203080018
:1003A0000A090402000103000000092111010001F3
:1003B0002236000705830308000A0904030002032C
:1003C0000000000921110100012222000705840319
:1003D00020000107050403200001120110010000A4
:1003E0000008EDFE01980101010200010631FF093C
:1003F00074A1010975150026FF009520750881027A
:100400000976150026FF00952075089102C00501A8
:100410000980A10185021601002637001A81002AF1
:10042000B700751095018100C0050C0901A1018577
:1004300003160100269C021A01002A9C02751095E1
:10044000018100C005010902A1010901A1000509FE
:1004500019012905150025019505750181029501F0
:10046000750381010501093009311581257F950248
:100470007508810609381581257F95017508810663
:10048000050C0A38021581257F950175088106C083
:10049000C005010906A101050719E029E715002596
:1004A00001950875018102950175088101050819FA
:1004B00001290595057501910295017503910105C5
:1004C00007190029FF150026FF0095067508810011
:1004D000C0636F6E73756D65723A20253034580AAB
:1004E0000073797374656D3A20253034580A000A18
:1004F000002530325820006B6579626F6172643A72
:1005000020004C45443A20253032580A0025583AFC
:100510002530386225730A000A2020303132333406
:100520003536370A00290A002575002F0025750089
:100530005D2800256400200025640020002564005B
:1005400020002564007C0025303258006D6F7573E3
:10055000656B6579205B62746E7C782079207620EB
:10056000685D287265702F61636C293A205B006DAD
:100570006B5F776865656C5F74696D655F746F5FED
:100580006D6178203D2025640A006D6B5F7768659A
:10059000656C5F6D61785F7370656564203D2025D3
:1005A000640A006D6B5F74696D655F746F5F6D6188
:1005B00078203D2025640A006D6B5F6D61785F7364
:1005C00070656564203D2025640A006D6B5F696E6F
:1005D00074657276616C203D2025640A006D6B5F46
:1005E00064656C6179203D2025640A006D6B5F773E
:1005F0006865656C5F74696D655F746F5F6D617868
:10060000203D2025640A006D6B5F776865656C5F2F
:100610006D61785F7370656564203D2025640A0014
:100620006D6B5F74696D655F746F5F6D6178203DA0
:100630002025640A006D6B5F6D61785F737065657E
:1006400064203D2025640A006D6B5F696E746572DD
:1006500076616C203D2025640A006D6B5F64656CDB
:100660006179203D2025640A000A00257500363A8C
:1006700020776865656C5F74696D655F746F5F6D29
:1006800061783A20000A00257500353A20776865C0
:10069000656C5F6D61785F73706565643A20000A10
:1006A00000257500343A2074696D655F746F5F6D65
:1006B00061783A20000A00257500333A206D617890
:1006C0005F73706565643A20000A00257500323A50
:1006D00020696E74657276616C286D73293A20000A
:1006E0000A00257500313A2064656C6179282A3149
:1006F000306D73293A20000A092D2056616C75650A
:1007000073202D0A004D3E004D25643E20003F0021
:100710007365742064656661756C740A00433E20DD
:100720000077686572652064656C74613A20637552
:1007300072736F723D25642C20776865656C3D256A
:10074000640A53656520687474703A2F2F656E2EA5
:1007500077696B6970656469612E6F72672F77695D
:100760006B692F4D6F7573655F6B6579730A000A4E
:10077000092D204D6F7573656B6579202D0A4553E2
:10078000432F713A09717569740A313A0964656CCD
:100790006179282A31306D73290A323A09696E74F9
:1007A000657276616C286D73290A333A096D617838
:1007B0005F73706565640A343A0974696D655F74C6
:1007C0006F5F6D61780A353A09776865656C5F6DB2
:1007D00061785F73706565640A363A0977686565A4
:1007E0006C5F74696D655F746F5F6D61780A0A7024
:1007F0003A097072696E742076616C7565730A646B
:100800003A097365742064656661756C74730A7562
:10081000703A092B310A646F776E3A092D310A70EC
:100820006775703A092B31300A7067646F776E3ADA
:10083000092D31300A0A7370656564203D206465B6
:100840006C7461202A206D61785F73706565642027
:100850002A2028726570656174202F2074696D6587
:100860005F746F5F6D6178290A003F004D3E200084
:10087000433E20004C25640A000A092D20436F6E78
:10088000736F6C65202D0A4553432F713A097175BA
:1008900069740A6D3A096D6F7573656B65790A0045
:1008A0000A092D204D61676963202D0A643A0964A5
:1008B000656275670A783A096465627567206D61DB
:1008C000747269780A6B3A096465627567206B65B2
:1008D00079626F6172640A6D3A09646562756720B6
:1008E0006D6F7573650A763A0976657273696F6E16
:1008F0000A733A097374617475730A633A09636F12
:100900006E736F6C65206D6F64650A302D343A0923
:100910006C61796572302D34284631302D4634298A
:100920000A506175733A09626F6F746C6F61646528
:10093000720A003F0074696D65725F7265616433AD
:100940003228293A202530346C580A006B657962C8
:100950006F6172645F69646C653A2025580A006BA8
:100960006579626F6172645F70726F746F636F6CD0
:100970003A2025580A00686F73745F6B6579626F5F
:100980006172645F6C65647328293A2025580A00F7
:100990000A092D20537461747573202D0A00474392
:1009A000433A20352E342E30204156522D4C4942A8
:1009B000433A20322E302E30204156525F4152436E
:1009C000483A20617672350A004F5054494F4E53D1
:1009D0003A204C554641204D4F5553454B455920E3
:1009E00045585452414B455920434F4E534F4C4567
:1009F00020434F4D4D414E4420343039360A004299
:100A000055494C443A206437336265646235202886
:100A100031353A35343A3435204A616E2031372049
:100A200032303231290A005649443A20307846455E
:100A3000454428742E6D2E6B2E29205049443A20AF
:100A40003078393830312850433938206B65796235
:100A50006F61726420636F6E7665727465722920AF
:100A60005645523A203078303130310A00444553EF
:100A7000433A20636F6E7665727473205043393841
:100A8000206B6579626F6172642070726F746F633E
:100A90006F6C20696E746F205553420A000A092D4D
:100AA0002056657273696F6E202D0A000A6D6F758E
:100AB00073653A206F66660A000A6D6F7573653A52
:100AC000206F6E0A000A6B6579626F6172643A206A
:100AD0006F66660A000A6B6579626F6172643A201C
:100AE0006F6E0A000A6D61747269783A206F6666EB
:100AF0000A000A6D61747269783A206F6E0A000A02
:100B000064656275673A206F6E0A000A64656275F3
:100B1000673A206F66660A000A0A626F6F746C6F2C
:100B2000616465722E2E2E2000433E2000001124A9
:100B30001FBECFEFDAE0DEBFCDBF04B603FE28C094
:100B400080915B0490915C04A0915D04B0915E047F
:100B50008730904BA740B04BD9F410925B041092B1
:100B60005C0410925D0410925E0414BE0FB6F894FB
:100B7000A895809160008861809360001092600069
:100B80000FBE1092010810920008E0E0F8E309950A
:100B900011E0A0E0B1E0E8EBFDE402C005900D92A9
:100BA000A833B107D9F724E0A8E3B1E001C01D9252
:100BB000AB35B207E1F70E94600B0C94DA260C9477
:100BC0000000FF93EF93E0913801F09139013097E5
:100BD00009F00995EF91FF910895FC01859180300E
:100BE00011F0EFDFFBCF0895FF27E0E230E247FF8F
:100BF0000CC0419597FF09C0EDE260957095809516
:100C00009095611D711D811D911D27FF02C02195C9
:100C100030E350E2AA27660F771F881F991FAA1F8B
:100C2000A41710F0A41B63955A95A9F7AA3008F0F1
:100C3000A95FA05DAF93F3956115710581059105DD
:100C400041F7ED3211F4EF93F395F21718F43F9357
:100C5000F395FBCF8F91B5DFFA95E1F70895E99110
:100C6000F9918591803021F0853219F0AADFF9CF12
:100C7000089520E0E89455915532C1F3503311F4B2
:100C8000689455915A3348F4505390F3220F022E32
:100C9000220F220F200D250FF4CF0EF421958991FC
:100CA0009991533619F3533729F1533559F1BC0152
:100CB00088279927E8945C3621F489919991689462
:100CC0005591543639F446EF7EF077FF0DC08FEF23
:100CD0009FEF0AC055374AE039F0583540E121F01E
:100CE000523642E009F00895FF93EF937DDFEF91D4
:100CF000FF91B7CFFF93EF93FC0181918030B9F35F
:100D000060DFFBCFFF93EF9368DFF1CFDF93CF93EB
:100D1000CDB7DEB72596A3DFCF91DF910895CF93AE
:100D2000C82F1F928F938BEC92E09F938F930E941A
:100D300086065C9A8FE99FE00197F1F700C00000FA
:100D40008C2F0E946F088FE99FE00197F1F700C098
:100D500000005C980F900F900F900F90CF91089526
:100D60001F93CF93DF931FEF0E945B08EC0111509C
:100D7000CF3F9FEFD90741F48FE99FE00197F1F74B
:100D800000C000001111F0CF5C9A85ED8A95F1F753
:100D900000005C98DF93CF9384EC92E09F938F9355
:100DA0000E9486060F900F900F900F90CE01DF915A
:100DB000CF911F910895EF92FF920F931F93CF93BE
:100DC000DF93539A549A519A5B9A5C9A599A0E946B
:100DD00045085C9A5B9820E52A95F1F75B9A8FEFBE
:100DE00090E722E0815090402040E1F700C00000F1
:100DF0008FE90E948F060E94B0068A3F910569F430
:100E00000E94B006803A910541F40E94B0068038F5
:100E1000910519F48CED92E002C082ED92E09F936F
:100E20008F930E9486060F900F9005EB12E086EAE2
:100E3000E82E82E0F82E8CE90E948F060E94B00610
:100E4000EC01CF3F8FEFD80729F4EBE3F1E08BE41F
:100E500091E02DC080913D0480FF0AC0DF93CF93C5
:100E60001F930F930E9486060F900F900F900F9084
:100E7000CA3FD10551F780E70E948F060E94B00655
:100E8000EC01CF3F8FEFD807B1F280913D0480FF96
:100E90000AC0DF93CF93FF92EF920E9486060F90D5
:100EA0000F900F900F90CA3FD10529F6CECF119227
:100EB0008E179F07E1F75C98DF91CF911F910F91FB
:100EC000FF90EF900895EF92FF920F931F93CF93AF
:100ED000DF930E945B08F82E082F192F0F3F8FEF2A
:100EE000180709F04EC080913A01882309F48FC099
:100EF00000E912E09FE7E92E92E0F92E8DE90E94C9
:100F00008F060E94B006EC01CF3F8FEFD80721F487
:100F100010923A0180E07BC080913D0480FF0AC0BE
:100F2000DF93CF931F930F930E9486060F900F902D
:100F30000F900F90CA3FD10559F780913A010E9456
:100F40008F060E94B006EC01CF3F8FEFD807B1F2B9
:100F500080913D0480FF10C0DF93CF9380913A01D0
:100F60001F928F93FF92EF920E9486060F900F9030
:100F70000F900F900F900F90CA3FD10509F0BECF90
:100F8000C7CF9F93FF928FE992E09F938F930E9428
:100F900086060F900F900F900F90E80183E0D69592
:100FA000C7958A95E1F76F2D67708C2F8F70F7FECC
:100FB00014C00E945212882319F1CF70DD27C55C3E
:100FC000DE4F0770112781E090E001C0880F0A957D
:100FD000EAF780959881892312C00E9452128111EC
:100FE0000FC0CF70DD27C55CDE4F0770112781E091
:100FF00090E001C0880F0A95EAF79881892B8883D1
:101000005C9A85ED8A95F1F700005C988F2DDF9151
:10101000CF911F910F91FF90EF900895E82FF0E08E
:10102000E55CFE4F8081089580FD02C090E701C01D
:1010300091E790933A0181FF05C090913A01946045
:1010400090933A0190913D0490FF0CC01F928F93B2
:1010500080E792E09F938F930E9486060F900F90F7
:101060000F900F9080913D0480FF0EC080913A0157
:101070001F928F9380E692E09F938F930E94860643
:101080000F900F900F900F90089583E38093CC0002
:101090001092CD00E9ECF0E080818069808380814E
:1010A00088608083EAECF0E08081806380835298DE
:1010B0005A9A7894089520914B0180914C0182179F
:1010C00059F030E0F901E35BFE4F80812F5F3F4F25
:1010D00020934B0190E008958FEF9FEF089590913A
:1010E000C80095FFFCCF8093CE0008951F920F9209
:1010F0000FB60F9211242F933F934F938F939F938B
:10110000EF93FF9380914C0190E09C012F5F3F4F44
:1011100040914B01421741F03091CE00FC01E35B5E
:10112000FE4F308320934C01FF91EF919F918F915F
:101130004F913F912F910F900FBE0F901F901895D8
:10114000809159030895CF93DF9300D01F92CDB7BC
:10115000DEB79C0180915204843019F593E09983A5
:101160003B832A839093E9008FEF9091E8008150B0
:1011700095FD06C095ED9A95F1F700008111F5CF28
:101180008091E80085FF0DC040E050E063E070E032
:10119000CE0101960E94160D8091E8008E77809313
:1011A000E8000F900F900F90DF91CF910895CF93AB
:1011B000DF9300D01F92CDB7DEB7209152042430C8
:1011C00031F522E02983805891099B838A8383E04B
:1011D0008093E9008FEF9091E800815095FD06C063
:1011E00095ED9A95F1F700008111F5CF8091E80017
:1011F00085FF0DC040E050E063E070E0CE01019655
:101200000E94160D8091E8008E778093E8000F9081
:101210000F900F90DF91CF910895209152042430C8
:10122000F1F422E02093E9002FEF3091E800215003
:1012300035FD06C035ED3A95F1F700002111F5CFE7
:101240002091E80025FF0BC040E050E065E070E031
:101250000E94160D8091E8008E778093E800089533
:10126000CF93DF9320915204243049F521E020935D
:10127000E90021E8215059F03091E80035FD07C020
:10128000EFE3F1E03197F1F700C00000F3CF2091D8
:10129000E80025FF14C0EC0140E050E068E070E099
:1012A0000E94160D8091E8008E778093E80088E018
:1012B000FE01A1E5B3E001900D928A95E1F7DF917F
:1012C000CF910895CF93C0914F02C1110BC00E94DE
:1012D0004F1E643C79408105910520F081E08093A8
:1012E0004F02C1E08C2FCF910895FF920F931F936F
:1012F000CF93DF93D82F0FB607FE83C0809152049F
:10130000843081F08091030190E0019620910501E5
:1013100030E0822393232091040130E08217930769
:1013200009F0CDC00E946209811110C080910301B3
:1013300090E001962091050130E0822393232091D3
:10134000040130E08217930709F0B9C00E94431EE0
:101350008C01C091E900CF709091EC00892F8170D1
:1013600090FD80E8C82B84E08093E90085E0F82EAA
:101370008091EB0085FD42C08091EB0080FF3EC074
:101380008091EE0087FF3AC08091040190910301A3
:10139000981709F457C09091E80095FF8EC0E0912E
:1013A0000101F0910201E80FF11D20818F5F909102
:1013B00005018923809304012093F1008091E800C6
:1013C00085FDE2CF8091E80080FFDECF8091E800CC
:1013D0008E778093E800F0920001D6CF80910301D0
:1013E00090E001962091050130E082239323209123
:1013F000040130E08217930709F44CC0CF70C0930A
:10140000E90040910301842F90E0019620910501AD
:1014100030E0822393232091040130E08217930768
:1014200009F450C0E0910101F0910201E40FF11DB7
:10143000D083809103018F5F909105018923809370
:10144000030140C08091E80085FF37C0D093F100D0
:1014500021E03091F3008091F20090E0932B892BF2
:1014600091F08091E80080FF0EC08091E80085FF38
:1014700003C01092F100F9CF8091E8008E7780933D
:10148000E800F0920001222309F4A8CFCF70C093A6
:10149000E90018C080910001882309F4AFCF0E94B1
:1014A000431E9C018017910711F4890161CF90912F
:1014B0000001915090930001F8CF20E0CACF4091F5
:1014C0000301B0CF80E0DF91CF911F910F91FF908A
:1014D000089580915104811104C00E94820F0C94E0
:1014E000DF0F0895109251040895089542E061ECD1
:1014F00081E00E948F0C42E061EC82E00E948F0C40
:1015000042E061EC83E00E948F0C42E261EC84E0F7
:101510000C948F0C80915404833009F453C030F440
:10152000813071F0823009F48CC008958A3009F45A
:1015300078C08B3009F45EC0893009F09AC020C0B1
:1015400080915304813A09F094C08091E800877F2C
:101550008093E8008091570490915804892B21F4DE
:1015600068E081E593E003C060E080E090E070E037
:101570000E94630D8091E8008B778093E8000895C6
:1015800080915304813209F074C080915704909186
:101590005804892B09F06DC08091E800877F809303
:1015A000E8008091E80082FD05C08091520481111D
:1015B000F8CF5FC08091F100809359038091E800DB
:1015C0008B7753C080915304813A09F052C08091C7
:1015D000570490915804892B09F04BC08091E80082
:1015E000877F8093E8008091E80080FFFCCF8091A6
:1015F000100136C0809153048132D9F5809157048F
:1016000090915804892BA9F58091E800877F8093F9
:10161000E8000E94C40C80915504809310010C9442
:10162000F51380915304813221F58091E800877F82
:101630008093E8000E94C40C8091560480935A0362
:10164000089580915304813AA1F48091E800877F46
:101650008093E8008091E80080FFFCCF80915A03DE
:101660008093F1008091E8008E778093E8000C94DD
:10167000C40C08958091590380935002109259032D
:101680000E9450120C94F5130C943A0B0E94D01D3A
:1016900080915004882329F00E94F91D81110C9437
:1016A000790C08950E940D1E809150028093590379
:1016B00008950C94520B08950C945B0B0C945B0BE7
:1016C000CF9384B7877F84BF0FB6F894A895809195
:1016D0006000886180936000109260000FBE90E00F
:1016E00080E80FB6F89480936100909361000FBE7C
:1016F00085E799E00E94A31D86E091E00E94E61034
:101700008AE093E00E94ED050E945E0B0E94A51105
:101710000E94820F0E94DF0F78940E94A71180918F
:101720005204843029F00E94CB100E945B0BF7CF4B
:1017300088EF92E00E94ED050E945C0B86EE92E03D
:101740000E94ED05C4E080915204853019F40E9496
:10175000460BF9CF0E94AB112091E4003091E500D7
:1017600080914D0290914E022817390709F468C004
:101770008091E4009091E50090934E0280934D0299
:101780000E946209882309F45BC08091520484306E
:1017900009F056C08091E9008F702091EC00922FE3
:1017A000917020FD90E8892BC093E9009091EB00A7
:1017B00090FF43C09091EE0097FF3FC090910401CD
:1017C00020910301291709F12091E80025FF1DC090
:1017D000E0910101F0910201E90FF11D30819F5F5D
:1017E000209105019223909304013093F100909190
:1017F000E80095FDE3CF9091E80090FFDFCF909156
:10180000E8009E779093E800D9CF9091F300209163
:10181000F20030E0392B232B81F09091E80090FF0B
:101820000CC09091E80095FF03C01092F100F9CF31
:101830009091E8009E779093E8008F708093E90084
:101840000E94CB1080CF292F332723303105C9F0D8
:1018500060F42130310581F02230310509F041C0BA
:1018600084E790E026E633E040C021323105E1F024
:101870002232310531F135C082E190E02AED33E0CA
:1018800034C099278130910549F028F0029749F535
:10189000E0E2F3E005C0E2E6F3E002C0E2E5F3E0F7
:1018A000849190E09F0121C064307105D0F4660FEF
:1018B000771FFB01EB5DFE4F2081318189E090E0D5
:1018C00014C06430710568F4FB01EE0FFF1FE35E86
:1018D000FE4F20813181FB01E75EFE4F808190E069
:1018E00004C080E090E020E030E0FA013183208302
:1018F000089580E189BD82E189BD09B400FEFDCF74
:101900008091D8008F7D8093D8008091E000826024
:101910008093E0008091E00081FDFCCF0895982F36
:10192000973068F59093E900981739F07091EC00C2
:101930002091ED005091F00003C0242F762F50E04D
:1019400021FD02C09F5FECCF3091EB003E7F3093D2
:10195000EB003091ED003D7F3093ED003091EB00D6
:1019600031603093EB007093EC002093ED005093C6
:10197000F0002091EE0027FDE5CF80E008958F7004
:101980008093E90081E008958091530487FF11C09E
:101990008091E80082FD05C0809152048111F8CF4A
:1019A00011C08091E8008B770BC08091520488238E
:1019B00049F08091E80080FFF8CF8091E8008E77B1
:1019C0008093E80008952091E4003091E50095E6C9
:1019D0004091EC00842F817040FF23C08091E8008B
:1019E00080FD1DC080915204882399F0853099F0C4
:1019F0008091EB0085FD11C04091E4005091E5001D
:101A00002417350729F3915011F09A01E1CF84E0B2
:101A1000089582E0089583E0089581E0089580E0CC
:101A200008954091E80042FFDDCF0895CF92DF9204
:101A3000EF92FF920F931F93CF93DF93EC018B01F3
:101A40007A010E94E30C811135C0E114F10439F0F0
:101A5000F70180819181081B190BC80FD91FC12C78
:101A6000D12C0115110529F18091E80085FD18C0E0
:101A70008091E8008E778093E8000E94CB10E114FB
:101A8000F10449F0F70180819181C80ED91ED182FD
:101A9000C08285E00FC00E94E30C882311F30AC0C6
:101AA00089918093F10001501109FFEFCF1ADF0AED
:101AB000D8CF80E0DF91CF911F910F91FF90EF90F1
:101AC000DF90CF9008952091590430915A04261741
:101AD000370748F06115710539F42091E8002E7739
:101AE0002093E80001C0B901FC0120E061157105F7
:101AF00079F1809152048823F1F18530F1F18091E0
:101B0000E80083FD3CC08091E80082FD2EC08091FA
:101B1000E80080FFEBCF2091F3008091F20090E08D
:101B2000922B6115710551F08830910538F421919F
:101B30002093F100615071090196F3CF21E00897DD
:101B400009F020E08091E8008E778093E800CECF06
:101B50002111CFCF0AC080915204882361F08530D3
:101B600061F08091E80083FD0AC08091E80082FF67
:101B7000F2CF80E0089582E0089583E0089581E047
:101B800008952091590430915A042617370748F0D8
:101B90006115710539F42091E8002E772093E80053
:101BA00001C0B901FC0120E06115710591F180913E
:101BB0005204882309F440C0853009F43FC0809165
:101BC000E80083FD3DC08091E80082FD2FC0809138
:101BD000E80080FFE9CF2091F3008091F20090E0CF
:101BE000922B6115710559F08830910540F42491CC
:101BF0002093F1003196615071090196F2CF21E0F6
:101C0000089709F020E08091E8008E778093E80043
:101C1000CBCF2111CCCF0AC080915204882361F030
:101C2000853061F08091E80083FD0AC08091E80072
:101C300082FFF2CF80E0089582E0089583E0089566
:101C400081E008951F93CF93DF93CDB7DEB7AA97B6
:101C50000FB6F894DEBF0FBECDBFE3E5F4E0809190
:101C6000F100819324E0EB35F207C9F70E948A0A5C
:101C70008091E80083FF2EC1809153049091540419
:101C8000492F50E04A30510508F024C1FA01EA5AC0
:101C9000FF4F0C94C026803821F0823809F01AC119
:101CA00008C080914F0490915004992389F082607C
:101CB0000FC0809157048F70873008F00BC180935C
:101CC000E9008091EB0085FB882780F91092E900FC
:101CD0009091E800977F9093E8008093F100109234
:101CE000F100D1C0282F2D7F09F0F4C0882319F00E
:101CF000823061F0EFC080915504813009F0EAC074
:101D0000933009F080E0809350042EC080915504F8
:101D100081112AC0809157048F702FEF280F263031
:101D200008F0D8C08093E9002091EB0020FF1CC090
:101D3000933021F48091EB00806214C09091EB000D
:101D400090619093EB0021E030E0A90102C0440FC4
:101D5000551F8A95E2F74093EA001092EA008091BD
:101D6000EB0088608093EB001092E9008091E8001E
:101D7000877F8093E8000E94C40CACC08111AAC088
:101D8000109155041F778091E3008078812B809318
:101D9000E3008091E800877F8093E8000E94C40CF4
:101DA0008091E80080FFFCCF8091E3008068809301
:101DB000E300111102C082E001C083E0809352046D
:101DC00089C08058823008F085C080915504909178
:101DD00056048C3D53E0950779F583E08A838AE2C7
:101DE00089834FB7F894DE01139620E03EE051E27C
:101DF000E32FF0E050935700E49120FF03C0E295F9
:101E0000EF703F5FEF708E2F90E0EA3010F0C796D2
:101E100001C0C0968D939D932F5F243149F74FBF2A
:101E20008091E800877F8093E8006AE270E0CE014D
:101E300001960E94630D16C060915704709158047A
:101E4000AE014F5F5F4F0E94230CBC01892B09F448
:101E500041C09091E800977F9093E80089819A8132
:101E60000E94C10D8091E8008B778093E80032C01A
:101E7000803881F58091E800877F8093E800809129
:101E80004E048093F1008091E8008E7772CF81112B
:101E900021C0809155049091560499270297D4F45B
:101EA0008091E800877F8093E800809155048093BB
:101EB0004E040E94C40C80914E04811106C0809192
:101EC000E30087FD02C081E001C084E080935204FA
:101ED0000E94760A8091E80083FF0AC08091E800A2
:101EE000877F8093E8008091EB0080628093EB0015
:101EF000AA960FB6F894DEBF0FBECDBFDF91CF918B
:101F00001F9108950E94F00F0E94F80FE0EEF0E09C
:101F1000808181608083E8EDF0E080818F7780832D
:101F200019BCA7EDB0E08C918E7F8C9380818F7E61
:101F300080831092510408950F931F93CF93DF93E2
:101F40000E94F00F0E94F80FC8EDD0E088818F77D3
:101F5000888388818068888388818F7D888319BC85
:101F60001092520410924E041092500410924F049A
:101F700000EE10E0F80180818B7F80838881816092
:101F8000888342E060E080E00E948F0CE1EEF0E0A8
:101F900080818E7F8083E2EEF0E0808181608083AB
:101FA000808188608083F80180818E7F8083888132
:101FB00080618883DF91CF911F910F910895E8EDA3
:101FC000F0E080818F7E8083E7EDF0E080818160AA
:101FD000808384E082BF81E0809351040C949C0F45
:101FE000E8EDF0E080818E7F80831092E20008951A
:101FF0001092DA001092E10008951F920F920FB62E
:102000000F9211242F933F934F935F936F937F937E
:102010008F939F93AF93BF93EF93FF938091E100D2
:1020200082FF0BC08091E20082FF07C08091E10037
:102030008B7F8093E1000E94CA108091DA0080FFBC
:102040001FC08091D80080FF1BC08091DA008E7F76
:102050008093DA008091D90080FF0DC080E189BDB6
:1020600082E189BD09B400FEFDCF81E08093520476
:102070000E94690A05C019BC109252040E94720A9B
:102080008091E10080FF19C08091E20080FF15C0BF
:102090008091E2008E7F8093E2008091E200806177
:1020A0008093E2008091D80080628093D80019BCB0
:1020B00085E0809352040E94440B8091E10084FFEC
:1020C00030C08091E20084FF2CC080E189BD82E1B4
:1020D00089BD09B400FEFDCF8091D8008F7D80932B
:1020E000D8008091E1008F7E8093E1008091E20032
:1020F0008F7E8093E2008091E20081608093E20015
:1021000080914E04882311F084E007C08091E300A1
:1021100087FD02C081E001C083E0809352040E94E9
:10212000590B8091E10083FF24C08091E20083FF7E
:1021300020C08091E100877F8093E10082E080935E
:10214000520410924E048091E1008E7F8093E10052
:102150008091E2008E7F8093E2008091E2008061B6
:102160008093E20042E060E080E00E948F0C0E94D9
:10217000750AFF91EF91BF91AF919F918F917F91E0
:102180006F915F914F913F912F910F900FBE0F90E4
:102190001F9018950895CF93809152048823A1F041
:1021A000C091E900CF709091EC00892F817090FD73
:1021B00080E8C82B1092E9008091E80083FD0E941E
:1021C000220ECF70C093E900CF91089590936003E1
:1021D00080935F030895E0915F03F091600330976F
:1021E00021F00190F081E02D099480E00895EF92B4
:1021F000FF920F931F93CF93DF93E0915F03F091D2
:1022000060033097B1F18C010280F381E02D0995D4
:1022100080913D0482FF2DC080FF04C087EF94E0D1
:102220000E94ED05E80118E081EFE82E84E0F82E29
:1022300080913D0480FF0BC088811F928F93FF9295
:10224000EF920E9486060F900F900F900F90115002
:1022500021961111EDCF80913D0480FF0AC08FEED1
:1022600094E0DF91CF911F910F91FF90EF900C942C
:10227000ED05DF91CF911F910F91FF90EF900895A1
:10228000E0915F03F0916003309721F00480F581C5
:10229000E02D09940895CF93DF9320915D03309151
:1022A0005E032817390709F190935E0380935D035D
:1022B000E0915F03F09160033097B9F0EC01068084
:1022C000F781E02D099580913D0482FF0EC080FFCB
:1022D0000CC0DF93CF9381EE94E09F938F930E9485
:1022E00086060F900F900F900F90DF91CF91089579
:1022F000CF93DF9320915B0330915C03281739075C
:1023000009F190935C0380935B03E0915F03F0918C
:1023100060033097B9F0EC010084F185E02D099558
:1023200080913D0482FF0EC080FF0CC0DF93CF93ED
:1023300081ED94E09F938F930E9486060F900F90FB
:102340000F900F90DF91CF9108950C9451120E943D
:102350003A1E0C94DB06BF92CF92DF92EF92FF926F
:102360000F931F93CF93DF9300D000D01F92CDB770
:10237000DEB70E94630702E613E0F12C8F2D0E9466
:102380000E08B82EF801C080C82639F4F3940F5F08
:102390001F4FF0E1FF12F2CF30C080913D0481FD6C
:1023A0000E946612D12CEE24E3948C2D8E21F9F03C
:1023B000D982FA8291E08B2D8E2109F490E09B83E3
:1023C0000E94431E8160782F9D838C8349815A81AE
:1023D0006B818D810E949C1249815A816B817C8125
:1023E0008D810E94BB1DF80180818E258083D3944E
:1023F000EE0CF8E0DF12D9CFC9CF8FEF89838A8343
:102400001B820E94431E8160782F9D838C834981AB
:102410005A816B818D810E949C120E94BA1D0E947C
:10242000E7200E94EB1090916103891741F10E940F
:10243000EB108093610390913D0492FF0EC090FFDA
:102440000CC01F928F9382E095E09F938F930E9420
:1024500086060F900F900F900F90809161030F9060
:102460000F900F900F900F90DF91CF911F910F91D0
:10247000FF90EF90DF90CF90BF900C94CC1D0F9009
:102480000F900F900F900F90DF91CF911F910F91B0
:10249000FF90EF90DF90CF90BF9008950C941408B8
:1024A00008950895CF93C62F0E940E0821E030E0D2
:1024B00002C0220F331FCA95E2F790E02823392388
:1024C00081E0232B09F480E0CF910895EF92FF92F1
:1024D0000F931F93CF93DF9388E195E00E94ED0562
:1024E000C0E0D0E08DE2E82E81E0F82E0DE015E0AE
:1024F0008C2F0E940E080E94A81DFF92EF921F923F
:102500008F93DF93CF931F930F930E94860621969C
:102510008DB79EB708960FB6F8949EBF0FBE8DBFBD
:10252000C031D10529F7DF91CF911F910F91FF9015
:10253000EF90089508950895CF93DF93CDB7DEB758
:102540002B970FB6F894DEBF0FBECDBF942F4F83ED
:10255000252F588769877A878B874A855B85452B26
:1025600031F02F3F31F481E09F3F19F403C081E047
:1025700001C080E080FD07C04F81588569857A855C
:102580008B850E94BB1DDE01119686E0FD01119234
:102590008A95E9F785E0FE01379601900D928A95BC
:1025A000E1F749815A816B817C818D819E810E94F6
:1025B0001D1A2B960FB6F894DEBF0FBECDBFDF916C
:1025C000CF910895CF93DF93882309F48FC0C82F4C
:1025D0008EE78C0F833018F5C23829F0C33831F0FC
:1025E000C4E0D7E405C0C2E0D9E302C0C1E0D3E54E
:1025F0000E94EB108C2309F079C08D2F0E94051DDD
:102600000E947D1D2FEF81EE94E02150804090408C
:10261000E1F700C000008D2F0E94221D10C08CEF3A
:102620008C0F813A20F080E58C0F8E3260F48C2F75
:102630000E94112481115AC08C2F0E94051DDF9128
:10264000CF910C947D1D80E28C0F883048F4C770C8
:1026500081E001C0880FCA95EAF70E94431DEFCFC1
:102660008BE58C0F833080F4C53A29F0C63A31F0FF
:1026700083E890E005C081E890E002C082E890E045
:10268000DF91CF910C944B1188E58C0F873170F559
:10269000C83A89F0C93A91F0CA3A99F0CB3AA1F018
:1026A000CC3AA9F0CD3AB1F0CE3AB9F0CF3AC1F078
:1026B00080E090E017C082EE90E014C089EE90E0D8
:1026C00011C08AEE90E00EC085EB90E00BC086EB67
:1026D00090E008C083EB90E005C084EB90E002C07E
:1026E00087EB90E0DF91CF910C947811DF91CF913F
:1026F0000895CF93DF93882309F454C09EE7980F81
:10270000933008F5823829F0833831F0C4E0D7E4FB
:1027100005C0C2E0D9E302C0C1E0D3E50E94EB10DE
:102720008C2309F43FC08D2F0E94051D0E947D1D42
:102730002FEF81EE94E0215080409040E1F700C0FF
:1027400000008D2F08C09CEF980F913A20F090E583
:10275000980F9E3218F40E94221D0DC090E2980F2F
:10276000983068F4877091E001C0990F8A95EAF774
:10277000892F0E94491DDF91CF910C947D1D9BE50F
:10278000980F933030F480E090E0DF91CF910C947B
:102790004B11885A873130F480E090E0DF91CF917F
:1027A0000C947811DF91CF910895882321F00E9435
:1027B000431D0C947D1D0895882321F00E94491D1E
:1027C0000C947D1D08950E94631D0E94321D0E947D
:1027D0007D1D0E948C210E945A2080E090E00E9482
:1027E0004B1180E090E00C9478110E94531D0C94E2
:1027F000E313CF92DF92EF92FF920F931F93CF9349
:10280000DF9300D000D01F92CDB7DEB76C010E94DD
:10281000CE1D811118C385E0F601DE0111960190ED
:102820000D928A95E1F7F60140815181238134812F
:102830002115310531F05F3F31F481E04F3F19F44C
:1028400003C081E001C080E080FDFDC2F601F2809E
:10285000E580E2948FE0E82249835A83FB82722F5D
:102860003D832C836F2D8D810E94811C8C010E94E1
:10287000801C0E94701BE12FE295EF708E2F90E07C
:10288000FC01E05AFF4F0C94C026812F807F1F70FF
:10289000882311F01295107FFF20B9F0112329F041
:1028A000812F0E94561D0E947D1D802F0F900F903A
:1028B0000F900F900F90DF91CF911F910F91FF908C
:1028C000EF90DF90CF900C94E212802F0E9479134A
:1028D000112309F4B8C2812F0E945C1D0F900F9044
:1028E0000F900F900F90DF91CF911F910F91FF905C
:1028F000EF90DF90CF900C947D1D812F807F1F7013
:10290000803211F01295107F002319F0013009F187
:102910002BC0FF20A9F0EE2059F1F1E0812FEF123A
:1029200028C00F900F900F900F900F90DF91CF91D4
:102930001F910F91FF90EF90DF90CF900C94661D48
:10294000EE2021F021E0E21609F47DC20E94691D0B
:102950004DC0FF20E9F085E08E1508F474C20E9496
:10296000401D812329F042C0FF20F1F1E11015C084
:10297000812F0F900F900F900F900F90DF91CF91BC
:102980001F910F91FF90EF90DF90CF900C94D51393
:1029900094E09E1508F457C229C0F601858180FF96
:1029A00013C08F708583E4CF003F09F489C108F01C
:1029B00055C180E4800F803208F459C1FF2009F42A
:1029C000EAC1EE2009F49AC1802F0E94E212093375
:1029D00009F0DAC1FFEF21EE84E0F15020408040A1
:1029E000E1F700C000002FC2E110D7C1812F59C10B
:1029F000812F86958695837019F08130B9F023C2B6
:102A0000FF2019F0C801937002C080E090E00F90A1
:102A10000F900F900F900F90DF91CF911F910F911A
:102A2000FF90EF90DF90CF900C944B11FF2019F0A6
:102A3000C801937002C080E090E00F900F900F905B
:102A40000F900F90DF91CF911F910F91FF90EF901A
:102A5000DF90CF900C947811802FFF2019F00E9406
:102A60006D1F02C00E94D51F0F900F900F900F9006
:102A70000F90DF91CF911F910F91FF90EF90DF901A
:102A8000CF900C945A20812F837009F070C0F11000
:102A9000DAC1202F229526952770220F220F602F52
:102AA0006F70862F90E0A0E0B0E06C017D01022EF7
:102AB00004C0CC0CDD1CEE1CFF1C0A94D2F704FFF2
:102AC00012C08FE090E0A0E0B0E004C0880F991F32
:102AD000AA1FBB1F2A95D2F7BC01CD016095709546
:102AE0008095909503C060E070E0CB011695169537
:102AF00013701230B1F040F56C297D298E299F2981
:102B0000113031F10F900F900F900F900F90DF91D7
:102B1000CF911F910F91FF90EF90DF90CF900C9489
:102B2000951B6C297D298E299F290F900F900F905E
:102B30000F900F90DF91CF911F910F91FF90EF9029
:102B4000DF90CF900C94AF1B0E94951BC701B6017C
:102B50000F900F900F900F900F90DF91CF911F91DA
:102B60000F91FF90EF90DF90CF900C947B1BFF2094
:102B700019F0812F817001C08695882309F463C103
:102B8000202F229526952770220F220F602F6F701D
:102B9000862F90E0A0E0B0E06C017D01022E04C021
:102BA000CC0CDD1CEE1CFF1C0A94D2F704FF12C0F3
:102BB0008FE090E0A0E0B0E004C0880F991FAA1F4A
:102BC000BB1F2A95D2F7BC01CD0160957095809509
:102BD000909503C060E070E0CB01169516951370D8
:102BE0001230B1F040F56C297D298E299F291130D2
:102BF00031F10F900F900F900F900F90DF91CF91C8
:102C00001F910F91FF90EF90DF90CF900C945C1C80
:102C10006C297D298E299F290F900F900F900F907E
:102C20000F90DF91CF911F910F91FF90EF90DF9068
:102C3000CF900C946E1C0E945C1CC701B6010F90D3
:102C40000F900F900F900F90DF91CF911F910F91E8
:102C5000FF90EF90DF90CF900C944A1C023F09F454
:102C60005EC008F449C0033F09F46CC0A7CE902FA2
:102C70009071E92E812F8F71FF2051F00E94E31B8C
:102C8000802FEE2019F08295807F73CE8F7071CEE9
:102C90000E94041C802FEE2019F08295807F01C0D5
:102CA0008F700F900F900F900F900F90DF91CF913A
:102CB0001F910F91FF90EF90DF90CF900C94DC1359
:102CC000FF20A9F0E4E0EE1508F4BDC0812F8F715C
:102CD0000F900F900F900F900F90DF91CF911F9159
:102CE0000F91FF90EF90DF90CF900C94291CF5E0AE
:102CF000FE1508F4A8C0EACFFF2099F0812F8F714C
:102D00000F900F900F900F900F90DF91CF911F9128
:102D10000F91FF90EF90DF90CF900C94E31BFF207A
:102D200069F3812F8F710F900F900F900F900F907C
:102D3000DF91CF911F910F91FF90EF90DF90CF9097
:102D40000C94041CFF2089F0812F8F710F900F903D
:102D50000F900F900F90DF91CF911F910F91FF90E7
:102D6000EF90DF90CF900C94CE1B0F900F900F90B0
:102D70000F900F90DF91CF911F910F91FF90EF90E7
:102D8000DF90CF900C94C91B033509F423CE073490
:102D900009F059C01FCEEE2021F2802F0F900F9026
:102DA0000F900F900F90DF91CF911F910F91FF9097
:102DB000EF90DF90CF900C947913412F4F70602FDC
:102DC000C6010E94E71E0F900F900F900F900F907A
:102DD000DF91CF911F910F91FF90EF90DF90CF90F7
:102DE0000C94CB1A01112FC0FF2069F10E94F5133A
:102DF0002FEF80E792E0215080409040E1F700C043
:102E000000000F900F900F900F900F90DF91CF91D7
:102E10001F910F91FF90EF90DF90CF900C94901E38
:102E2000412F4F70602FC6010F900F900F900F90A1
:102E30000F90DF91CF911F910F91FF90EF90DF9056
:102E4000CF900C94EA1E0F900F900F900F900F9060
:102E5000DF91CF911F910F91FF90EF90DF90CF9076
:102E600008951F93CF93DF9300D000D01F92CDB76A
:102E7000DEB7942F4983252F5A836B837C838D8300
:102E80004C815D81452B31F02F3F31F481E09F3F34
:102E900019F403C081E001C080E0182F117080FD9B
:102EA00031C049815A816B817C818D810E94811C56
:102EB000292F22952F702C3030F42A30A0F4225084
:102EC000223030F022C02C30C9F02F30B9F01DC0B4
:102ED000853A28F48430C0F4823028F415C090E29A
:102EE000980F983088F0883E30F4803E68F4845023
:102EF000813A58F409C0803F41F406C093FB112782
:102F000010F903C010E001C011E0812F0F900F9065
:102F10000F900F900F90DF91CF911F910895CF9355
:102F2000DF9300D000D01F92CDB7DEB70F900F9087
:102F30000F900F900F90DF91CF910895CF93DF9373
:102F400000D000D000D0CDB7DEB726960FB6F894EB
:102F5000DEBF0FBECDBFDF91CF9108951F93CF93FA
:102F6000DF93C091720316E080917303C81799F044
:102F7000D0E01C9FF0011D9FF00D1124EC58FC4F78
:102F80004081518162817381848195810E949E1765
:102F90002196C770E9CFDF91CF911F91089540919D
:102FA000A4035091A5036091A6037091A70380919B
:102FB000A8039091A9030C949E170F931F93CF938E
:102FC000DF938091A90382958F7009F05DC0809195
:102FD000A603882309F458C08091720310917303EB
:102FE0006091A4037091A503C091A703D091A80399
:102FF00091E06F3F09F090E0292F06E0811709F476
:1030000043C0209721F07F3F21F030E003C031E042
:1030100001C0322F90E030FD34C0089FF001099FBD
:10302000F00D1124DF01AC58BC4F11963C91119763
:10303000371327C03C91361324C012963C91129747
:1030400031111FC013964D915C9114974C1B5D0B71
:10305000483C5105B0F48091A9038F708061809342
:10306000A903E758FC4F80818F708061808384EAD8
:1030700093E00E94F913DF91CF911F910F910C946F
:10308000AE1701968770BACFDF91CF911F910F9144
:1030900008959F92AF92BF92CF92DF92EF92FF92EC
:1030A0000F931F93CF93DF93CDB7DEB761970FB622
:1030B000F894DEBF0FBECDBF8C0185E0F801DE01C4
:1030C0001D9601900D928A95E1F7F801408151819A
:1030D000F280C380D4809091A4036091A5032091D5
:1030E000A7033091A8032115310531F06F3F31F46A
:1030F00081E09F3F19F403C081E001C080E0F82F18
:10310000F1709F2E80FD52C184EAA82E83E0B82E74
:10311000E090A603F601E21BF30BEE2009F4E8C0F1
:103120008091A903E83CF10508F0A4C0282F207F76
:1031300009F053C0561313C0491311C0EF2CF110FE
:103140000EC08F7080618093A9030E94CF17C501C4
:103150000E94F9138091A903F80185835BC1C11412
:10316000D10431F05F3F31F481E04F3F19F403C0E7
:1031700081E001C080E080FD03C081E08F2502C0B6
:1031800080E090E0F82FF170EF2E80FF1CC080915E
:1031900072032091730336E0821709F418C190E09E
:1031A000389FF001399FF00D1124EC58FC4F6181DC
:1031B000561306C06081461303C06281F61203C035
:1031C00001968770E9CFEF2CFF2009F423C180918D
:1031D000A90381608093A90362C0561306C04913F6
:1031E00004C0F11002C0F801A7C04D875E87FF86BA
:1031F0007C2DD98AC88A6F2D89890E94311788232E
:1032000099F1FF2089F12091A903822F82958F7077
:1032100090E0029774F08091A4039091A5039887A1
:103220008F831986DB86CA862C87CE0107960E947B
:10323000F91386E0F801A4EAB3E001900D928A95B3
:10324000E1F70E94DD170E94CF1711C0561749F110
:103250004D875E87FF867C2DD98AC88A6F2D898924
:103260000E94311781112CC0C8010E94F913EE246D
:10327000E394D0C0282F207F49F77C2DD98AC88AB3
:103280006F2D89890E948F1784EA93E00E94F913B9
:1032900086E0F50111928A95E9F70E94CF17E12C9B
:1032A000B9C04913D5CFF110D3CFF8018583C80138
:1032B0000E94F91386E0F50111928A95E9F7AAC0F8
:1032C000FF2091F22091A903822F82958F7090E0C8
:1032D00002970CF4AECF8091A4039091A5039A833A
:1032E00089831B82DD82CC822E83CE0101969FCF03
:1032F000E83CF10508F04BC0EF2CFF2009F4B4CFF7
:10330000561330C049132EC02091A90320FD21C0BF
:10331000822F82958F70482F50E041155105C9F0DA
:10332000F80125834F30510541F08F5F982F92951A
:10333000907F822F8F70892B8583C8010E94F9139B
:1033400086E0F801A4EAB3E001900D928A95E1F7D6
:103350002AC086E0F801A4EAB3E001900D928A95B4
:10336000E1F758C04D875E87FF867C2DD98AC88AD1
:103370006F2D89890E94311781115BCF8091A9033C
:1033800081608093A903C8010E94F91343C07C2D7A
:10339000D98AC88A6F2D89890E948F1786E0F50126
:1033A00011928A95E9F70E94CF1734C0FF2009F4E3
:1033B0005BCF4D875E87FF867C2DD98AC88A6F2DAB
:1033C00089890E943117882309F44ECF32CF7C2D92
:1033D000D98AC88A6F2D89890E94811C292F22953C
:1033E0002F70223028F49F7039F0811105C00BC076
:1033F000243028F49F7049F4805E883020F0C801A2
:103400000E94F9139E2CE92C05C0F8019581907F4C
:1034100099F7F9CF8E2D61960FB6F894DEBF0FBEE7
:10342000CDBFDF91CF911F910F91FF90EF90DF9073
:10343000CF90BF90AF909F9008951F93CF93DF934D
:10344000CDB7DEB72C970FB6F894DEBF0FBECDBF59
:103450004F83588769877A878B879C87CE01079629
:103460000E9449188823D1F09F8188852A853B8551
:10347000232B31F08F3F31F481E09F3F19F403C0DB
:1034800081E001C080E080FD47C04F81588569859B
:103490007A858B859C850E949E173EC086E0FE0142
:1034A0003796DE01119601900D928A95E1F7FF8122
:1034B000E8856A857B856115710531F0EF3F31F450
:1034C00081E0FF3F19F403C081E001C080E080FD8E
:1034D00023C02091730330E0C901019687709927BA
:1034E0004091720350E084179507F1F1F983EA8364
:1034F0007D836C8396E0929FD001939FB00D112441
:10350000AC58BC4FFE01319601900D929A95E1F7AF
:10351000809373030E94AE1716E08091720390911E
:103520007303891771F1189FC00111248C589C4FA7
:103530000E944918882329F1E09172031E9FF0012F
:103540001124EC58FC4F4081518162817381848148
:1035500095810E949E178091720390E0019687707A
:10356000992780937203D9CF0E94F51310927303A9
:1035700010927203E4EAF3E086E0DF011D928A957F
:10358000E9F72C960FB6F894DEBF0FBECDBFDF91E2
:10359000CF911F910895DF92EF92FF920F931F93A7
:1035A000CF93DF93FC01892B09F488C0E12CF12C27
:1035B000DD24D394EF0121968491853709F460C00E
:1035C00058F4843708F04EC0843008F068C0813069
:1035D000D1F0823071F172C0883709F45BC050F4C9
:1035E000863709F453C0873709F068C08E2D0E94D2
:1035F000501D52C09CE7980F903708F05FC08F773E
:103600000E9479134EC08F010E5F1F4FFE018491FF
:1036100090E2980F983050F48770FD2D01C0FF0F95
:103620008A95EAF78F2F0E94561D15C00E94E2125C
:1036300014C08F010E5F1F4FFE01849190E2980F1E
:10364000983068F48770FD2D01C0FF0F8A95EAF766
:103650008F2F0E945C1D0E947D1DE80122C00E94E8
:103660007913FBCFCF010296FE01C491CC2361F008
:10367000EFE9FFE03197F1F700C00000C150F6CF4D
:10368000CF010296FE01F490EC010BC00E94401D98
:10369000E82E07C00E94531D0E947D1D02C00E949B
:1036A000E2128F2D882341F0EFE9FFE03197F1F727
:1036B00000C000008150F6CFFE017CCFDF91CF919A
:1036C0001F910F91FF90EF90DF90089560932A046F
:1036D00070932B0480932C0490932D040C94CB1D99
:1036E000089560932E0470932F0480933004909378
:1036F00031040C94CA1D0F931F9300912E04109156
:103700002F042091300430913104602B712B822BD7
:10371000932B60932E0470932F0480933004909326
:1037200031041F910F910C94CA1D0F931F930091A8
:103730002E0410912F042091300430913104602325
:1037400071238223932360932E0470932F0480931C
:103750003004909331041F910F910C94CA1D0F9364
:103760001F9300912E0410912F042091300430916A
:103770003104602771278227932760932E0470936A
:103780002F0480933004909331041F910F910C9477
:10379000CA1D60E070E0CB010C94661B0F931F9371
:1037A00041E050E060E070E08A019B0104C0000F3E
:1037B000111F221F331F8A95D2F7C901B8011F912B
:1037C0000F910C94661B0F931F9341E050E060E053
:1037D00070E004C0440F551F661F771F8A95D2F70B
:1037E00080912A0490912B04A0912C04B0912D0477
:1037F0008A019B01082B192B2A2B3B2BC901B801ED
:103800001F910F910C94661B0F931F9341E050E0A2
:1038100060E070E004C0440F551F661F771F8A9553
:10382000D2F7409550956095709580912A049091BB
:103830002B04A0912C04B0912D048A019B01082334
:1038400019232A233B23C901B8011F910F910C941E
:10385000661B0F931F9341E050E060E070E004C0EE
:10386000440F551F661F771F8A95D2F780912A044F
:1038700090912B04A0912C04B0912D048A019B01FE
:10388000082719272A273B27C901B8011F910F9143
:103890000C94661B0F931F9300912A0410912B0424
:1038A00020912C0430912D04602B712B822B932BB3
:1038B0001F910F910C94661B0F931F9300912A0484
:1038C00010912B0420912C0430912D04602371233E
:1038D000822393231F910F910C94661B0F931F93C8
:1038E00000912A0410912B0420912C0430912D0476
:1038F00060277127822793271F910F910C94661BD5
:1039000008958F929F92AF92BF92DF92EF92FF92B3
:103910000F931F93CF93DF9300D000D01F92CDB7AA
:10392000DEB76B837C838D838A018C819D81892B9B
:1039300031F01F3F31F481E04F3F19F403C081E0C3
:1039400001C080E080FF03C080E090E04DC08B812B
:103950008823D1F180902A0490902B04A0902C040D
:10396000B0902D0480912E0490912F04A0913004EA
:10397000B0913104882A992AAA2ABB2A8FE1E82E1D
:10398000F12CD501C4010E2C04C0B695A7959795CE
:1039900087950A94D2F780FD06C081E0E81AF10805
:1039A00080F7D12C07C0DE2CB8018E2D0E94BF1EDF
:1039B000019799F388E0189FF0011124E655FC4F18
:1039C000E00FF11DD08209C088E0189FF00111249A
:1039D000E655FC4FE00FF11DD08009831A83698101
:1039E0007A818D2D0E94BF1E0F900F900F900F9027
:1039F0000F90DF91CF911F910F91FF90EF90DF908B
:103A0000BF90AF909F908F900895209111013091B9
:103A10001201F90132969FEF40E05191851789F02C
:103A20009F3F19F4511101C0942F4F5F4630A9F701
:103A30009F3F39F0F901E90FF11D97FDFA95828357
:103A400008950895E0911101F09112019F012A5FFC
:103A50003F4F9281891301C012823196E217F3071A
:103A6000C1F7089581E090E0E0911101F091120119
:103A7000E80FF91F1082019688309105A9F7089583
:103A800080913C04089590913C04892B80933C04E0
:103A90000895809590913C04892380933C04089577
:103AA00080933C04089510923C04089590913B0447
:103AB000892B80933B040895809590913B04892342
:103AC00080933B04089510923B0408958093320440
:103AD000089510923204089580911101909112017D
:103AE000FC0131969C01285F3F4F80E0919191113C
:103AF0008F5FE217F307D1F70895E0911101F0917C
:103B0000120180913C048083E0911101F091120137
:103B1000908180913B04892B80838091320488239B
:103B200061F0E0911101F09112019081892B808365
:103B30000E946C1D811110923204809111019091AC
:103B400012010C94F7109093390180933801089575
:103B50008295982F937344E0949F900111248C7C5C
:103B600086958695282B822F8575880F2A7A26952B
:103B7000822B08950895CF93DF9300D000D01F9239
:103B8000CDB7DEB70F900F900F900F900F90DF9191
:103B9000CF910895089508950C944E1280E00895F1
:103BA00080915204843021F110923E0420E488E197
:103BB00090E00FB6F894A895809360000FBE209314
:103BC000600083B7817F846083BF83B7816083BFD8
:103BD0007894889583B78E7F83BF0FB6F894A895A5
:103BE00080916000886180936000109260000FBE39
:103BF0000895CF930E949A120E9463070E949B121D
:103C0000C0E08C2F0E940E08811104C0CF5FC0312C
:103C1000C1F701C081E0CF9108950E9450120C9429
:103C2000F5131F920F920FB60F9211248F939F934B
:103C3000AF93BF9380913E04811113C080913F04E4
:103C400090914004A0914104B09142044196A11D7D
:103C5000B11D80933F0490934004A0934104B0931E
:103C60004204BF91AF919F918F910F900FBE0F9023
:103C70001F90189582E084BD93E095BD9AEF97BDA3
:103C800080936E0008952FB7F89480913F0490912F
:103C90004004A0914104B09142042FBF08952FB772
:103CA000F89460913F047091400480914104909198
:103CB00042042FBF08959C014FB7F89480913F04B0
:103CC00090914004A0914104B09142044FBF821BE7
:103CD000930B089578941F920F920FB60F921124B0
:103CE0008F939F93AF93BF9380913F049091400433
:103CF000A0914104B09142040196A11DB11D809391
:103D00003F0490934004A0934104B0934204BF91B8
:103D1000AF919F918F910F900FBE0F901F901895AC
:103D20000E94820FF89487E797E7909301088093A9
:103D3000000887E090EBDC0180935B0490935C04C7
:103D4000A0935D04B0935E049CE088E10FB6F89404
:103D5000A895809360000FBE90936000FFCFE82F7E
:103D6000F0E088E0989FE00DF11D1124E052FE4F35
:103D70008491982F92959F708F7097700895CF932C
:103D8000C82FCB010E94AF1E40E1949F90011124E7
:103D9000282B203831051CF080E090E016C0977089
:103DA000E92FF0E098E0C99FE00DF11D112494E0A7
:103DB000EE0FFF1F9A95E1F78F70E80FF11DEE0FE0
:103DC000FF1FE052FF4F85919491CF91089580E0BD
:103DD00090E0089508958091450480FF0BC06091A4
:103DE000160185E0689FB00111247595679575955A
:103DF00067952BC081FF09C06091160185E0689F1F
:103E0000B00111247595679520C082FF07C06091AD
:103E1000160185E0689FB001112417C090914604F7
:103E20009923D1F060911501961788F7209116011A
:103E300085E0289F90011124929FA001939F500D2F
:103E4000112470E0CA010E94AC266038710540F46C
:103E50006115710519F406C065E070E0862F0895BC
:103E60008FE7089581E008958091450480FF08C0A0
:103E70006091140170E0759567957595679521C0FF
:103E800081FF06C06091140170E07595679519C0B7
:103E900082FF04C06091140170E010C0909146044C
:103EA000992399F0609113019617A0F7809114015E
:103EB000899FC001112470E00E94AC266038710512
:103EC00040F46115710519F406C061E070E0862FB9
:103ED00008958FE7089581E00895803F21F40E94BE
:103EE000EB1E819504C0813F29F40E94EB1E809354
:103EF00049040895823F21F40E94EB1E819504C07D
:103F0000833F29F40E94EB1E809348040895893F63
:103F100019F40E94341F05C08A3F31F40E94341FF7
:103F2000819580934A0408958B3F21F40E94341FA9
:103F3000819504C08C3F29F40E94341F80934B0468
:103F40000895843F21F480914704816017C0853F24
:103F500021F480914704826011C0863F21F4809152
:103F6000470484600BC0873F21F480914704886038
:103F700005C0883F31F480914704806180934704F5
:103F800008958D3F21F48091450481600BC08E3FE0
:103F900021F480914504826005C08F3F29F480910F
:103FA00045048460809345040895803F39F48091EE
:103FB000490487FF6CC01092490469C0813F29F40D
:103FC000809149041816BCF362C090914804823F66
:103FD00029F497FF5CC01092480459C0833F19F43C
:103FE0001916CCF354C0893F41F480914A04181645
:103FF0000CF04DC010924A044AC08A3F29F48091C7
:104000004A0487FF44C0F6CF8B3F39F480914B04BC
:1040100087FF3DC010924B043AC08C3F29F4809139
:104020004B041816BCF333C0843F21F4809147043D
:104030008E7F17C0853F21F4809147048D7F11C08A
:10404000863F21F4809147048B7F0BC0873F21F48A
:1040500080914704877F05C0883F31F480914704F1
:104060008F7E8093470413C08D3F21F480914504D7
:104070008E7F0BC08E3F21F4809145048D7F05C05B
:104080008F3F29F4809145048B7F80934504809174
:10409000480481110EC08091490481110AC08091A9
:1040A0004A04811106C080914B04811102C0109214
:1040B0004604089580913D0483FF7EC08CE495E022
:1040C0000E94ED05809147041F928F9387E495E04D
:1040D0009F938F930E94860685E495E00E94ED05EC
:1040E00080914804282F082E000C330B3F938F93A8
:1040F00082E495E09F938F930E94860680E495E08A
:104100000E94ED0580914904282F082E000C330BE6
:104110003F938F938DE395E09F938F930E94860644
:104120008BE395E00E94ED0580914A04282F082E2C
:10413000000C330B3F938F9388E395E09F938F930D
:104140000E94860686E395E00E94ED0580914B046F
:10415000282F082E000C330B3F938F9383E395E0B9
:104160009F938F930E94860680E395E00E94ED0561
:10417000809146041F928F938DE295E09F938F93D9
:104180000E9486068BE295E00E94ED058091450431
:104190001F928F9388E295E09F938F930E948606EB
:1041A00085E295E00E94ED058DB79EB74C960FB65F
:1041B000F8949EBF0FBE8DBF87E494E00E9440112B
:1041C0000E94431E909344048093430408951F93D8
:1041D000CF93DF9380914304909144040E945B1E2F
:1041E000AC0190914604992321F02091170130E011
:1041F00006C0209118018AE0289F900111244217DF
:10420000530708F485C080914804C0914904D091B7
:104210004A0410914B04811107C0C11175C0D1111E
:1042200073C0111171C074C09F3F19F09F5F9093CC
:104230004604181624F40E94EB1E809348048091D3
:10424000480487FF05C00E94EB1E819580934804B7
:104250001C1624F40E94EB1E8093490480914904AB
:1042600087FF05C00E94EB1E8195809349046091F1
:104270004804662331F1C0914904CC2311F1062E84
:10428000000C770B880B990B0E94B32523E333E3D3
:1042900043E35FE30E9417260E947B256093480456
:1042A0006C2FCC0F770B880B990B0E94B32523E35F
:1042B00033E343E35FE30E9417260E947B2560936C
:1042C00049041D1624F40E94341F80934A048091EF
:1042D0004A0487FF05C00E94341F819580934A04D9
:1042E000111624F40E94341F80934B0480914B04D8
:1042F00087FF05C00E94341F819580934B04DF9196
:10430000CF911F910C945A209F3F09F08FCFA0CFDF
:10431000DF91CF911F910895E7E4F4E085E0DF019C
:104320001D928A95E9F7109246041092450408956B
:104330008FE697E00E94ED051F9281E08F931F9218
:1043400085E08F9381E297E09F938F930E9486068A
:104350000F900F900F900F900F900F900895833053
:10436000E9F128F4813061F0823009F10895853057
:1043700009F462C008F449C0863009F474C0089595
:1043800080911801262F30E0280F311D2F3F310575
:1043900024F4680F6093180103C08FEF8093180115
:1043A000809118011F928F938AE596E072C08091E8
:1043B0001701262F30E0280F311D2F3F310524F43F
:1043C000680F6093170103C08FEF809317018091EE
:1043D00017011F928F9388E496E05BC080911601CD
:1043E000262F30E0280F311D2F3F310524F4680FB0
:1043F0006093160103C08FEF809316018091160120
:104400001F928F9385E396E044C080911501262F7B
:1044100030E0280F311D2F3F310524F4680F6093E1
:10442000150103C08FEF80931501809115011F9234
:104430008F9380E296E02DC080911401262F30E00A
:10444000280F311D2F3F310524F4680F60931401AC
:1044500003C08FEF80931401809114011F928F93FA
:1044600087E096E016C080911301262F30E0280FD8
:10447000311D2F3F310524F4680F6093130103C0F1
:104480008FEF80931301809113011F928F938CEE15
:1044900095E09F938F930E9486060F900F900F9048
:1044A0000F900895833081F128F4813059F08230E3
:1044B000D1F00895853009F449C0B8F1863009F487
:1044C00056C0089580911801681720F4861B8093C8
:1044D000180102C010921801809118011F928F9349
:1044E0008DED95E054C080911701681720F4861B6C
:1044F0008093170102C010921701809117011F923B
:104500008F938BEC95E043C080911601681720F4DF
:10451000861B8093160102C010921601809116012D
:104520001F928F9388EB95E032C080911501681738
:1045300020F4861B8093150102C010921501809112
:1045400015011F928F9383EA95E021C08091140199
:10455000681720F4861B8093140102C01092140186
:10456000809114011F928F938AE895E010C080918A
:104570001301681720F4861B8093130102C0109268
:104580001301809113011F928F938FE695E09F9303
:104590008F930E9486060F900F900F900F900895B2
:1045A000CF93C82F1F928F9384E798E09F938F93A8
:1045B0000E94860681E090E0A0E0B0E0BC01CD0161
:1045C00004C0660F771F881F991FCA95D2F70E94F3
:1045D000711B0F900F900F900F90CF910C94F513CB
:1045E000CF93873288F58E3108F00BC18E3009F4F5
:1045F00087C0D8F4873009F460C08B3009F44FC00D
:10460000863009F002C180913D04817F8E7F8093C6
:104610003D0489E798E00E94ED0589E29BE00E9455
:10462000ED0581E080934D0446C0863109F4B0C0A9
:1046300020F4803109F47AC0E8C0893109F491C0CE
:104640008B3109F449C0E1C0883349F150F4893213
:1046500009F4D5C0853309F4D2C0873209F0D5C03A
:10466000CEC0833409F4CBC028F48A3308F4CDC01B
:104670008953C8C0883409F0C8C00E94F51388E186
:104680009BE00E94ED052FEF83ED90E321508040E9
:104690009040E1F700C000000E94901E0CC080EA2C
:1046A00098E041C08FEF9AE00E94ED0580913D04B3
:1046B000816080933D04C1E0ADC080913D04C82F6E
:1046C000C17080FFEFCF8BE09BE00E94ED058091F1
:1046D0003D04817F8E7F3FC090913D0491FBCC27AC
:1046E000C0F981E0C827892FC0FB81F980933D0480
:1046F000CC2319F082EF9AE029C084EE9AE013C02F
:1047000090913D0492FBCC27C0F981E0C827892F06
:10471000C0FB82F980933D04CC2319F085ED9AE02B
:1047200015C085EC9AE00E94ED05C5CF90913D043F
:1047300093FBCC27C0F981E0C827892FC0FB83F900
:1047400080933D04CC2351F089EB9AE00E94ED0563
:1047500080913D04816080933D045CC08CEA9AE0C6
:10476000E2CF8DE99AE00E94ED058DE69AE00E9485
:10477000ED0587E29AE00E94ED058FEF99E00E9437
:10478000ED0589EC99E00E94ED058EE999E0CBCF2B
:1047900080E999E00E94ED050E94EB101F928F9333
:1047A00086E799E09F938F930E948606809110017F
:1047B0001F928F938FE599E09F938F930E948606B7
:1047C00080915A031F928F938CE499E09F938F936B
:1047D0000E9486060E944F1E9F938F937F936F9334
:1047E00085E399E09F938F930E9486068DB79EB7CD
:1047F00042960FB6F8949EBF0FBE8DBF5CCF80E08F
:1048000001C08D510E94D02256CF83E399E00E94CF
:10481000ED05C0E08C2FCF91089580E008950C94B1
:104820000D240F931F93CF93C82F80914D04813097
:10483000B1F020F0823009F45BC052C160E070E05A
:104840008CE090E00E945212892BC9F4E091110192
:10485000F09112018081843409F044C110C060E0FD
:1048600070E08CE090E00E9452128C01892B39F4A8
:10487000E0911101F09112018081843461F48C2F58
:104880000E940F24811104C08C2F0E94F0222EC0A0
:1048900081E090E02BC08C2F0E940D24811124C157
:1048A000C431E1F070F4CB3081F0C031D1F40E941A
:1048B00098218CE698E00E94ED0582E080934D04FB
:1048C00013C1C93259F0C83361F489E798E00E94F6
:1048D000ED0580E798E00E94ED0506C110924D04B9
:1048E00004C08AE698E00E94ED05802F8170FFC029
:1048F000C43228F5CE3108F0C1C0CB30A1F1D0F4DC
:10490000C73009F0D3C08EE18093180182E3809311
:1049100017018AE08093160184E18093150188E0F5
:104920008093140188E28093130180E197E00E9454
:10493000ED05BFC0C33149F1C431C1F0B7C0CB34BC
:1049400009F4A9C028F4C93289F0C83361F0AEC0B7
:10495000C13509F49EC0C23509F499C0CE3409F0BE
:10496000A5C06AE09EC00E949821A3C080914C041B
:10497000882319F010924C049CC08DE197E00E94AE
:10498000ED0581E080934D04B2C087EF96E00E9470
:10499000ED0585EE96E00E94ED05809118011F92CD
:1049A0008F9382EE96E09F938F930E94860680EE0F
:1049B00096E00E94ED058EEC96E00E94ED05809158
:1049C00017011F928F938BEC96E09F938F930E9419
:1049D000860689EC96E00E94ED058AEB96E00E943F
:1049E000ED05809116011F928F9387EB96E09F93C0
:1049F0008F930E94860685EB96E00E94ED0584EA7F
:104A000096E00E94ED05809115011F928F9381EA37
:104A100096E09F938F930E9486068FE996E00E940E
:104A2000ED058AE896E00E94ED05809114011F9241
:104A30008F9387E896E09F938F930E94860685E880
:104A400096E00E94ED058EE696E00E94ED058091CD
:104A500013011F928F938BE696E09F938F930E9492
:104A6000860689E696E00E94ED058DB79EB74896CA
:104A70000FB6F8949EBF0FBE8DBF1BC0CE51EC2F5A
:104A8000F0E0E25DFE4F808180934C0412C061E053
:104A900003C061E006C06AE080914C040E94AF212F
:104AA00008C080914C040E94522203C08EE097E01F
:104AB00013C080914C04882369F01F928F9388E083
:104AC00097E09F938F930E9486060F900F900F9010
:104AD0000F9004C085E097E00E94ED0581E007C0DB
:104AE00010924D0480E003C001E010E0FECECF91B3
:104AF0001F910F9108950E9482256894B1110C9422
:104B0000112608950E94F62588F09F5798F0B92F36
:104B10009927B751B0F0E1F0660F771F881F991FF2
:104B20001AF0BA95C9F714C0B13091F00E9410265E
:104B3000B1E008950C941026672F782F8827B85F6E
:104B400039F0B93FCCF3869577956795B395D9F74A
:104B50003EF490958095709561957F4F8F4F9F4F54
:104B60000895E89409C097FB3EF490958095709560
:104B700061957F4F8F4F9F4F9923A9F0F92F96E9A9
:104B8000BB279395F695879577956795B795F1111E
:104B9000F8CFFAF4BB0F11F460FF1BC06F5F7F4FBB
:104BA0008F4F9F4F16C0882311F096E911C07723CD
:104BB00021F09EE8872F762F05C0662371F096E8D6
:104BC000862F70E060E02AF09A95660F771F881FA5
:104BD000DAF7880F9695879597F9089557FD9058BD
:104BE000440F551F59F05F3F71F04795880F97FBB1
:104BF000991F61F09F3F79F087950895121613066B
:104C00001406551FF2CF4695F1DF08C01616170699
:104C10001806991FF1CF86957105610508940895CE
:104C2000E894BB2766277727CB0197F908950E9460
:104C30002A260C949B260E948D2638F00E949426EA
:104C400020F0952311F00C9484260C948A261124CC
:104C50000C9411260E94EE2570F3959FC1F3950FD9
:104C600050E0551F629FF001729FBB27F00DB11DF0
:104C7000639FAA27F00DB11DAA1F649F6627B00D80
:104C8000A11D661F829F2227B00DA11D621F739F69
:104C9000B00DA11D621F839FA00D611D221F749F77
:104CA0003327A00D611D231F849F600D211D822FBE
:104CB000762F6A2F11249F5750409AF0F1F08823E5
:104CC0004AF0EE0FFF1FBB1F661F771F881F915012
:104CD0005040A9F79E3F510580F00C9484260C9417
:104CE00011265F3FE4F3983ED4F386957795679558
:104CF000B795F795E7959F5FC1F7FE2B880F911D3C
:104D00009695879597F9089597F99F6780E870E0E1
:104D100060E008959FEF80EC089500240A94161631
:104D2000170618060906089500240A941216130699
:104D3000140605060895092E0394000C11F4882327
:104D400052F0BB0F40F4BF2B11F460FF04C06F5F43
:104D50007F4F8F4F9F4F089597FB072E16F40094B7
:104D600007D077FD09D00E94C62607FC05D03EF487
:104D7000909581959F4F0895709561957F4F089507
:104D8000EE0FFF1F0590F491E02D0994AA1BBB1BA9
:104D900051E107C0AA1FBB1FA617B70710F0A61B3B
:104DA000B70B881F991F5A95A9F780959095BC015C
:084DB000CD010895F894FFCF36
:104DB8000551020000FFA00830090D09D708A30813
:104DC8000133042808140A321E404D362291044447
:104DD800040E04EC0378039103AA03C30300010241
:084DE800030405060708090099
:00000001FF
